:0A00000075817F7401F58F02000E78
:10000B000208AF75F15490000074F2F0A37407F07E
:10001B0090000274F2F0A37407F090000474F2F0F5
:10002B00A37407F012013BC209120FC1C2B6C2B5CD
:10003B00C2B712109E1210CF121100D2B6D2B5D287
:10004B00B7C215C216C2177590FB75A0FFD2B4C20A
:10005B000FC212C210C213C211C214C200C202C21A
:10006B0004C201C203C205C206C207C208C209C24A
:10007B000AC20BD227D228D229C22DC22EC22FC21E
:10008B003FD221D222D223C23CC23DC23ED218D291
:10009B0019D21A12012712087DD22AD22BD22C7513
:1000AB0064C87566C87568C8755B64755E80755C79
:1000BB0064755F80755D6475608075410075420085
:1000CB00753900753A0012047C1204B41204EC85E5
:1000DB00414385424412052C1201271201271201BC
:1000EB002712113112032D12033F12035112047CFC
:1000FB001204B41204EC1204981204D012027312FC
:10010B00029A1202C112052C120557120582020027
:10011B00EC783279FF0000D9FCD8F822786479FFAB
:10012B000000D9FCD8F822781E7996D9FED8FA228D
:10013B00C2B6D2B5D2B7120127120127C2B6C2B5C9
:10014B00D2B7120127120127C2B6C2B5C2B712012C
:10015B0027120127120127120127C2B6C2B5D2B747
:10016B00120127120127C2B6D2B5D2B7120127123C
:10017B000127D2B6D2B5D2B712012712012712012D
:10018B002712012722E627F5280809E637F52978F3
:10019B002822C3E697F5280809E697F5297828223F
:1001AB008628872A08098629872B120230782D2268
:1001BB00862D08862E08862F088630872A09872BDE
:1001CB001201D37828792F22753100753210120263
:1001DB00151201E6120209D532F422C3E52F952A36
:1001EB00E530952BE5319400500122E52F952AF54A
:1001FB002FE530952BF530E5319400F53122B3E541
:10020B002833F528E52933F52922C3E52D33F52DC0
:10021B00E52E33F52EE52F33F52FE53033F530E5AD
:10022B003133F53122E528852AF0A4F52D85F02E02
:10023B00E529852BF0A4F52F85F030E529852AF0EB
:10024B00A4252EF52EE52F35F0F52FE5303400F5EE
:10025B0030E528852BF0A4252EF52EE52F35F0F56E
:01026B002F63
:10026C00E5303400F53022120A26200C0122C20C93
:10027C0030000C1205AD1205D61205F9D21222125D
:10028C00060912061B120644D20F1203C122120ACF
:10029C007A200D0122C20D30020C12065C1206856A
:1002AC001206A8D213221206B81206CA1206F3D2EC
:1002BC001012040122120ACE200E0122C20E3004AA
:1002CC000C12070B120734120757D21422120767AD
:1002DC001207791207A2D211120441222081102098
:1002EC000110B200D201200005C218D2242222C271
:1002FC00012222208010200310B202D2032002051A
:10030C00C219D2252222C2032222209010200510CD
:10031C00B204D205200405C21AD2262222C205221A
:10032C00223000012220A708203C07D23CD2122206
:10033C00C23C223002012220A708203D07D23DD228
:10034C001322C23D223004012220A708203E07D2EE
:10035C003ED21422C23E22308410200910202D05DA
:10036C00D218D20922D209C22D22C20922223085EA
:10037C0010200A10202E05D219D20A22D20AC22E1F
:10038C0022C20A2222308210200B10202F05D21AF2
:10039C00D20B22D20BC22F22C20B22222086122079
:1003AC000612B221D206D22DC21BC21CC230C231DF
:1003BC0022C2062222201817C215C2B6202108120A
:1003CC000B438843894422120BB88843894422C2C8
:1003DC0015D2B6A841A9428843894422208712200D
:1003EC000712B222D207D22EC21DC21EC232C23393
:1003FC0022C2072222201917C216C2B520220812C7
:10040C000C658845894622120CDA8845894622C239
:10041C0016D2B5A83BA93C884589462220831220D8
:10042C000812B223D208D22FC21FC220C234C23546
:10043C0022C2082222201A17C217C2B72023081280
:04044C000D87884749
:10045000894822120DFC8847894822C217D2B7A8C2
:100460003DA93E88478948227A0FC294D2A2A2A110
:1004700033C933C9C2A2DAF2F8D29422D2947A05EF
:1004800074E0C2A2C2943392A0D2A2DAF512046838
:10049000883F894053400F22D2947A0574E8C2A263
:1004A000C2943392A0D2A2DAF5120468883B893C48
:1004B000533C0F22D2947A0574F0C2A2C2943392B4
:1004C000A0D2A2DAF51204688839893A533A0F2289
:1004D000D2947A0574F8C2A2C2943392A0D2A2DA5E
:1004E000F5120468883D893E533E0F2285393385D5
:1004F0003A347833853F3785403879371201908612
:10050000F008E6120ED9F54285F04122853F338589
:1005100040347833853937853A38793712019D86EA
:10052000F008E6120EE6F54285F04122A843A94400
:10053000D295D2A4E944707A08C2A3C296339297A6
:10054000D2A3DAF57A08E8C2A3C296339297D2A36F
:10055000DAF5C295D29622A845A946D295D2A4E949
:1005600044F07A08C2A3C296339297D2A3DAF57AFE
:1005700008E8C2A3C296339297D2A3DAF5C295D205
:100580009622A847A948D295D296E944707A08C223
:10059000A3C2A4339297D2A3DAF57A08E8C2A3C221
:1005A000A4339297D2A3DAF5C295D2A422200F01E8
:1005B00022D215C20FC21BC21CC230C231755B648D
:1005C000755E80120B2290000085824F85835075E6
:1005D00049FF754A1422854F82855083A94212082B
:1005E00020A3A841120830A385824F858350854FF0
:1005F000558550568843894422D5490C7549FFD505
:100600004A06C200D22AC2182220120122C2129027
:10061000000085824F858350D22A22302A1D854FC3
:100620008285508312085BA312086CA385824F85D4
:10063000835088708971886A896B22A86AA96B883F
:1006400070897122E555B58212E556B5830D3024C7
:1006500008D212120609D22A22C22A22201001220E
:10066000D216C210C21DC21EC232C233755C64757E
:100670005F80120B2D90283C858251858352754BEB
:10068000FF754C1422855182855283A93C120820A3
:10069000A3A83B120830A385825185835285515708
:0506A000855258884559
:1006A500894622D54B0C754BFFD54C06C202D22B81
:1006B500C2192220130122C21390283C858251853C
:1006C5008352D22B22302B1D8551828552831208ED
:1006D5005BA312086CA3858251858352887089714A
:1006E500886C896D22A86CA96D8870897122E5577F
:1006F500B58212E558B5830D302508D2131206B818
:10070500D22B22C22B2220110122D217C211C21FC5
:10071500C220C234C235755D64756080120B389095
:100725005078858253858354754DFF754E14228507
:100735005382855483A93E120820A3A83D12083090
:10074500A385825385835485535985545A8847898F
:100755004822D54D0C754DFFD54E06C204D22CC28C
:100765001A2220140122C214905078858253858361
:1007750054D22C22302C1D85538285548312085B5C
:10078500A312086CA3858253858354887089718868
:100795006E896F22A86EA96F8870897122E559B597
:1007A5008212E55AB5830D302608D214120767D296
:1007B5002C22C22C220000D2B3000000000000C28F
:1007C500B3220000D2B3000000000000A2B4C2B3FF
:1007D500227E027A08EE3392B1FE1207BADAF622C9
:1007E500AE837A08EE3392B1FE1207BADAF6AE821C
:1007F5007A08EE3392B1FE1207BADAF622E9FE7AEA
:1008050008EE3392B1FE1207BADAF622E8FE7A084C
:10081500EE3392B1FE1207BADAF622D2B2C2B012A4
:1008250007D61207E5120802D2B022D2B2C2B01220
:1008350007D61207E5120811D2B0227E037A08EE18
:100845003392B1FE1207BADAF6227A081207C7EE1A
:1008550033FEDAF8F422D2B2C2B01208401207E52C
:1008650012084FF9D2B022D2B2C2B0120840120714
:10087500E512084FF8D2B0227587907589227598D0
:1008850050758C38758A38C0D043D008781479648F
:100895007A197B327C197D02D0D0756400756600AB
:1008A500756800D28CD2A9D2AF22C0E0C0D043D0A7
:1008B50008DD557D02D83F781912092212096B12FD
:1008C50009B412036312037A1203911202E81202A9
:1008D500FF1203160564E564120EA9F5640566E5C5
:1008E50066120EA9F5660568E568120EA9F568DCBD
:1008F500057C19120912D904A95BD20CDA04AA5C89
:10090500D20DDB04AB5DD20ED0D0D0E03230150273
:10091500B2B6301602B2B5301702B2B722300001B6
:10092500222084041203A82220861C200627D21226
:10093500D206D227756400756500D224C218C21B81
:10094500C21CC230C23122C206302709C2278564C3
:100955006512095B2222E565B42803020968500384
:08096500C22422D22422300238
:10096D0001222085041203E82220871C200727D2AC
:10097D0013D207D228756600756700D225C219C239
:10098D001DC21EC232C23322C207302809C22885B9
:10099D0066671209A42222E567B428030209B15043
:1009AD0003C22522D2252230040122208204120402
:1009BD00282220831C200827D214D208D22975683A
:1009CD0000756900D226C21AC21FC220C234C235B8
:1009DD0022C208302909C2298568691209ED22222F
:1009ED00E569B428030209FA5003C22622D2262251
:1009FD00E582C4540FF9E583C46922B48003020A69
:100A0D001B500B75F0038475F002A424102275F0B1
:100A1D00058475F003A42432223000012230180120
:100A2D002220210122853982853A831209FD301B4E
:100A3D000EF55EF4120A08120EC6F55BC21C2220DA
:100A4D001C10D21CB55E03D21B225003C23922D218
:100A5D00392220390CB55E03D21B22500122D21B44
:100A6D0022B55E03D21B225003D21B22223002017B
:100A7D00223019012220220122853B82853C8312DE
:100A8D0009FD301D0EF55FF4120A08120EC6F55C55
:100A9D00C21E22201E10D21EB55F03D21D2250038E
:100AAD00C23A22D23A22203A0CB55F03D21D22500F
:100ABD000122D21D22B55F03D21D225003D21D2269
:100ACD002230040122301A012220230122853D8289
:100ADD00853E831209FD301F0EF560F4120A0812CF
:100AED000EC6F55DC22022202010D220B56003D2A3
:100AFD001F225003C23B22D23B22203B0CB5600388
:100B0D00D21F22500122D21F22B56003D21F2250C4
:100B1D0003D21F222290000074F2F0A37407F0227A
:100B2D0090000274F2F0A37407F02290000474F2A6
:100B3D00F0A37407F02230210122853982853A8392
:100B4D001209FD30301CF56175F080846006120CC1
:100B5D0029020B64120BED900000E539F0A3E53A84
:100B6D00F022203119D231B56106D230120BB822E4
:100B7D005006C236120BB822D236120BB8222036CE
:100B8D0015B56106D230120BB8225004120BB822E3
:100B9D00D230120BB822B56106D230120BB82250EA
:100BAD0006D230120BB822120BB822900000E0F5DD
:100BBD0082900001E0F5831209FD75F080846010CC
:0C0BCD00900000E0F533900001E0F534EA
:100BD900120C2F22900000E0F537900001E0F53863
:100BE900120BF322853937853A3879377533007511
:100BF9003408753500753600783312019D8637083B
:100C090086387937857033857134753500753600C6
:100C1900783312019D86F008E6120EE6F9A8F02253
:100C2900853933853A34753500753600783375372B
:100C390000753808793712019D8633088634753571
:100C49000075360078338570378571387937120128
:100C59009086F008E6120ED9F9A8F0223022012276
:100C6900853B82853C831209FD30321CF56275F0A3
:100C790080846006120D4B020C86120D0F90000243
:100C8900E53BF0A3E53CF022203319D233B56206E7
:100C9900D232120CDA225006C237120CDA22D237BB
:100CA900120CDA22203715B56206D232120CDA227A
:100CB9005004120CDA22D232120CDA22B56206D2B0
:100CC90032120CDA225006D232120CDA22120CDA63
:100CD90022900002E0F582900003E0F5831209FDFD
:100CE90075F080846010900002E0F533900003E015
:100CF900F534120D5122900002E0F537900003E01F
:100D0900F538120D1522853B37853C38793775330F
:100D190000753408753500753600783312019D86E3
:100D2900370886387937857033857134753500759C
:100D39003600783312019D86F008E6120EE6F9A80E
:100D4900F022853B33853C347535007536007833A0
:100D5900753700753808793712019D86330886344E
:100D69007535007536007833857037857138793770
:100D790012019086F008E6120ED9F9A8F022302364
:100D89000122853D82853E831209FD30341CF563BD
:100D990075F080846006120E6D020DA8120E319056
:100DA9000004E53DF0A3E53EF022203519D235B522
:100DB9006306D234120DFC225006C238120DFC22F1
:100DC900D238120DFC22203815B56306D234120D23
:100DD900FC225004120DFC22D234120DFC22B56300
:100DE90006D234120DFC225006D234120DFC221206
:100DF9000DFC22900004E0F582900005E0F58312D5
:100E090009FD75F080846010900004E0F5339000CE
:0E0E190005E0F534120E7322900004E0F53768
:100E2700900005E0F538120E3722853D37853E38AC
:100E370079377533007534087535007536007833A2
:100E470012019D8637088638793785703385713466
:100E5700753500753600783312019D86F008E61265
:100E67000EE6F9A8F022853D33853E3475350075C9
:100E770036007833753700753808793712019D8643
:100E870033088634753500753600783385703785B5
:100E97007138793712019086F008E6120ED9F9A851
:100EA700F022B4C8012250012274C822B4320122B0
:100EB7005003743222B4C8012250012274C822B4EC
:100EC7001001225003741022B4C801225001227469
:100ED700C822B40F0122500122740F75F0FF22B40B
:100EE7000F0122500122740075F00022120F937433
:100EF700A0F9120F60120FAFE572F9120F60120F0F
:100F0700AFE573F9120F60120FAF120F9374A1F9C7
:100F1700120F60120FAF120F53120FAF120F85226D
:100F2700E9FA120F9374A0F9120F60120FAFE5726E
:100F3700F9120F60120FAFE573F9120F60120FAFBE
:100F4700EAF9120F60120FAF120F8522D2917808BB
:100F5700120FB5E933F9D8F8227808E9339291F9F5
:100F6700120FB5D8F6227B80DB02800E120F937426
:100F7700A0F9120F60120FAF40EE120F8522C29137
:100F870000D292000000000000D29122D29100D23C
:100F970092000000000000C291000000000000C2A3
:100FA7009222C291120FB522D291120FB5220000E0
:100FB700D292000000A291C292222084292009FA2D
:100FC700C2B6C2B5C2B7120FF012102A12106412BD
:100FD7000127120127120127120127D2B6D2B5D253
:100FE700B7D209020FC1C2092290000075491975CD
:100FF7004A018583728582737900120F27120F6D5C
:10100700A38583728582737900120F27120F6DA350
:10101700858255858356D549D9754919D54AD3123D
:10102700116B2290283C754B19754C01858372858D
:1010370082737900120F27120F6DA3858372858241
:10104700737900120F27120F6DA385825785835876
:10105700D54BD9754B19D54CD312118C229050789A
:10106700754D19754E018583728582737900120F4C
:1010770027120F6DA38583728582737900120F275C
:10108700120F6DA385825985835AD54DD9754D1990
:10109700D54ED31211AD221211CE90000085837266
:1010A700858273120EF3E9F9120820A385837285EE
:1010B7008273120EF3E9F8120830A3E555B582DD05
:1010C700E556B583D8D22A221211E990283C8583A8
:1010D70072858273120EF3E9F9120820A3858372D1
:1010E700858273120EF3E9F8120830A3E557B5822B
:1010F700DDE558B583D8D22B22121204905078859B
:101107008372858273120EF3E9F9120820A385838F
:1011170072858273120EF3E9F8120830A3E559B508
:1011270082DDE55AB583D8D22C2220A533201801B9
:101137002220190122201A01223000012230020147
:101147002230040122203F1BD23FD215D216D217DC
:1011570012121F121254121289D2B6D2B5D2B72266
:10116700C23F2222907850A95585837285827312D7
:101177000F27120F6DA3A956858372858273120FED
:1011870027120F6D22907852A95785837285827333
:0E119700120F27120F6DA3A95885837285824F
:1011A50073120F27120F6D22907854A959858372F7
:1011B500858273120F27120F6DA3A95A8583728535
:1011C5008273120F27120F6D2290785085837285D6
:1011D5008273120EF38955A3858372858273120E6D
:1011E500F3895622907852858372858273120EF3A5
:1011F5008957A3858372858273120EF389582290CD
:101205007854858372858273120EF38959A3858379
:1012150072858273120EF3895A2212116B900000A7
:1012250012085B858372858273E9F9120F27120F05
:101235006DA312086C858372858273E8F9120F27F6
:10124500120F6DA3E555B582D7E556B583D22212A7
:10125500118C90283C12085B858372858273E9F9AD
:10126500120F27120F6DA312086C85837285827386
:10127500E8F9120F27120F6DA3E557B582D7E55888
:10128500B583D2221211AD90507812085B85837216
:10129500858273E9F9120F27120F6DA312086C8569
:1012A5008372858273E8F9120F27120F6DA3E55932
:1012B500B582D7E55AB583D222464C414D45204BE0
:1012C5004E4F425245434F524445522D43332D4DC7
:1012D5004F44554C45204555524F205241434B20D4
:1012E50056455253494F4E202D203230313120562C
:1012F500455253494F4E20312E3030202863296204
:081305007920616D70657265CD
:00000001FF
